:100000000C9445040C9489040C9489040C94890480
:100010000C9489040C9489040C9489040C9489042C
:100020000C9489040C9489040C9458100C942A1193
:100030000C9489040C9489040C9489040C9489040C
:100040000C9489040C9434250C9489040C94890430
:100050000C9489040C94C71E0C9489040C94890494
:100060000C9489040C9489040C9489040C948904DC
:100070000C9489040C9489040C9489040C948904CC
:100080000C9489040C9489040C9489040C948904BC
:100090000C9489040C9489040C9489040C948904AC
:1000A0000C9489040C9489040C948904EE062807A6
:1000B0003A075C0774077A07800786078C07920760
:1000C00097079D07C707CC07D107E8079711B91114
:1000D000A712B911A712FE112112A71276128912C6
:1000E0005815581587158715BD15DD150E170E17F0
:1000F000E8150E1798169816FF160E170E17081704
:10010000A516A516A516A516A516A516A516A51617
:10011000A516A516A516A516A516A516A516A51607
:10012000B716C416CB16D216DC1602E002E2012E78
:10013000022E02E10002E002E102E20001E001E140
:1001400001E20002E002E3016402640002E002E373
:100150000001E001E30001E10137023702E101386B
:10016000023801E10125022502E10001E101370227
:100170003702E10138023801E10107020702E1001C
:1001800001350235012002200002E302E102E30210
:10019000E102E302E102E302E102E302E102E3023F
:1001A000E102E302E102E302E102E302E102E3022F
:1001B000E102E302E102E302E102E302E102E3021F
:1001C000E102E302E102E302E102E302E102E3020F
:1001D000E102E302E102E302E102E302E102E302FF
:1001E000E102E302E102E302E102E302E102E302EF
:1001F000E102E302E102E302E102E302E102E302DF
:10020000E102E302E102E302E102E302E102E302CE
:10021000E102E302E102E302E102E302E102E302BE
:10022000E10001E301E10001E10136023602E101F2
:1002300038023801E10126022602E10001E101371E
:10024000023702E10138023801E10126022602E10B
:100250000001E10136023602E10138023801E10114
:1002600025022502E10001E10137023702E10138F0
:10027000023801E20125022502E20001E101370214
:100280003702E10138023801E10130023002E100B9
:1002900002E002E2013002300002E002E20001E08E
:1002A00001E20001E10131023102E10029002B00ED
:1002B000E200E100354100001E00140004001D7141
:1002C0000E304E001F001A0016001B0003304C00B9
:1002D0002000080007000600E0022A0021001500A7
:1002E0000900190000304B00220017000A00050029
:1002F00000004A000230E3000000E20000004D0070
:100300000B30E7000000E6000000500023001C0056
:100310000B00110000004F00240018000D00100019
:100320003177520025000C000E0036002E7F2C0085
:10033000260012000F003700E108280027001300F4
:1003400033003871E10451002D002F003474E500B2
:1003500030410000650001000100010001000000C3
:100360003A00350031000100010001003B00350278
:100370002102350001004C003C001E02240622022E
:10038000010001003D002D022402240401000100AF
:100390003E00010037001104000001003E00010092
:1003A00000000100000001003F000100000001000A
:1003B000000068003F0024062402240400004500D9
:1003C0004000220425021104310269004100230487
:1003D000260201001F020100420035002504010031
:1003E00001000100430035022604010001306A00CB
:1003F00044001E0231000100010000000100010064
:1004000001000100010000000100010001000100E5
:10041000010001000100F400F200FB0001000100F6
:100420000100F000F100FA00010001000100F500F8
:10043000F300FC00010001000100F900FA00F600E1
:1004400000000100010001000000010000000100A7
:1004500001000100000001000000AC0001000100EB
:10046000010001000000AB000100010001000100DB
:100470000100A90001000100010001000100AE001F
:1004800001000100010001005000A800010001006E
:10049000010052005100AA0001000100010001000A
:1004A0004F000000010001000100010001000000F8
:1004B0000100010001000100010001000100010034
:1004C0000100010001000100010001000100010024
:1004D0000100010001000100010001000100010014
:1004E0000100010001000100000001000100010005
:1004F00000000100000001000730010000000100C1
:1005000000000100083005300A3001000000010041
:100510000C300D30043001000100010001000630F4
:1005200001000100010001000100010001000100C3
:1005300001000100010001000100010001000100B3
:1005400001000100010001000100000001000100A4
:100550000100010001000000010001000100010094
:100560000100010001000100500001000100010034
:1005700001005200510001000100010001000100D2
:100580004F00010001000100010001000100010015
:100590000000010001000100000001000000010056
:1005A0000100010000000100000001003F002402E2
:1005B00024022202000001004000240021001E004D
:1005C000270001004100250022001F003700010024
:1005D00042002600230020003600010043003002C4
:1005E00030000100270201004400450038000100EE
:1005F0000100000001000100E1000100E000000036
:10060000010001000100010001003D0001000100A6
:10061000010001000100E0000100010001000100F3
:1006200001002C00010001000100010001003C005C
:10063000010001000100010000003A00010001007A
:100640000000010000003B0001000100000001006B
:100650000000010001000100010001000000010094
:100660000100010001000100010001000100010082
:100670000100010001000100010001000100010072
:100680000100010001000100010001000130010032
:1006900001000100010001000100000016034500F7
:1006A000720067006F0044006F0078002000450072
:1006B0005A00000016034500720067006F004400F6
:1006C0006F007800200045005A0000000403090470
:1006D00009026D00040100A0FA09040000010301F1
:1006E0000100092111010001223F000705810308D3
:1006F000000A09040100010301020009211101009F
:1007000001224D000705820308000A0904020001C6
:1007100003000000092111010001223600070583B2
:100720000308000A09040300010300000009211165
:100730000100012239000705840310000112011095
:100740000100000008EDFE07130100010200010591
:10075000010906A101050719E029E7150025019502
:100760000875018102050819012905950575019192
:1007700002950175039101050719002977150025D8
:1007800001957875018102C005010980A1018502EA
:1007900016010026B7001A01002AB700751095014E
:1007A0008100C0050C0901A1018503160100269CEA
:1007B000021A01002A9C02751095018100C00501F2
:1007C0000902A1010901A100050919012905150066
:1007D00025019505750181029501750381010501CA
:1007E000093009311581257F950275088106093880
:1007F0001581257F950175088106050C0A380215BB
:1008000081257F950175088106C0C005010906A1F3
:1008100001050719E029E7150025019508750181F3
:1008200002950175088101050819012905950575CD
:100830000191029501750391010507190029FF1522
:100840000025FF950675088100C00000000000002B
:100850000000000000010204060A0F17202C3A4A8B
:100860005D71879DB3C7DAE9F5FCFFFCF5E9DAC7EE
:10087000B39D87715D4A3A2C20170F0A06040201C6
:100880000000000000000000000011241FBECFEF98
:10089000DAE0DEBFCDBF04B603FE24C08091FD01C7
:1008A0009091FE01A091FF01B09100028730904B22
:1008B000A740B04BB9F41092FD011092FE011092C6
:1008C000FF011092000214BE84B7877F84BF88E1C5
:1008D0000FB6F89480936000109260000FBEE0E0C5
:1008E000FFE3099511E0A0E0B1E0E6EFFDE402C00E
:1008F00005900D92A433B107D9F711E0A4E3B1E05C
:1009000001C01D92AD3FB107E1F70E949C0D0C9410
:10091000F9260C9400001092B9008AE08093B80088
:10092000089594EA9093BC009091BC0097FFFCCF8F
:100930009091B900987F983021F0903111F081E0CA
:1009400008958093BB0084E88093BC008091BC0034
:1009500087FFFCCF8091B900887F883111F0803407
:1009600071F780E0089584E98093BC008091BC0019
:1009700084FDFCCF08958093BB0084E88093BC0085
:100980008091BC0087FFFCCF9091B900987F81E0F7
:10099000983209F480E0089584E88093BC00809147
:1009A000BC0087FFFCCF8091BB00089580910101BE
:1009B000811115C080E40E9491048093010181118E
:1009C0000CC082E10E94BB0480930101811105C02B
:1009D0008FEF0E94BB04809301010E94B30484B195
:1009E000807F84B985B1807F85B98AB1837F8AB9D8
:1009F0008BB1837F8BB93E98469808950E949106EB
:100A0000809301010E94D60480B38C7080BB81B3B7
:100A1000836F81BBA5E3B1E0E3E4F1E08EE08E0FEC
:100A200011921D928E13FCCF0C947B06BF92CF9235
:100A3000DF92EF92FF920F931F93CF93DF938091FA
:100A40000101882379F0809134018F5F8093340114
:100A5000811108C00E94910680930101811102C09A
:100A60000E94230605E311E0C0E0D0E0DD24D3942A
:100A700082E0C82EEE24E394F12CC730D10500F5B6
:100A800080910101811164C080E40E9491048093EF
:100A90000101811112C082E10E94BB048093010117
:100AA00081110BC0C7010C2E01C0880F0A94EAF710
:100AB00080950E94BB04809301010E94B30448C04A
:100AC000CA30A1F028F4C83059F0C93061F005C02F
:100AD000CC3089F070F0CD3089F0209A289810C081
:100AE000219A29980DC0229A2A980AC0239A2B98F5
:100AF00007C0529A01C0539A5B9802C03E9A46982A
:100B000090EA9A95F1F79FB1799902C082E001C00D
:100B100080E091709D25982B7C9902C084E001C0F3
:100B200080E0892B7D9902C038E001C030E0832B42
:100B30007E9902C020E101C020E0822B9FB19095F8
:100B4000991F9927991F9295990F907E892B0FC015
:100B500080910101811149C080E40E949104809339
:100B60000101882379F1B12C0E94B3048B2DF80187
:100B70009081981719F08083C09200010E94D604DA
:100B800021960F5F1F4FCE30D10509F076CF8091AF
:100B90000001882361F1815080930001882339F09E
:100BA0008FE99FE00197F1F700C0000020C0A3E4A7
:100BB000B1E0E5E3F1E0CF01825F91919D938E1367
:100BC000FCCF15C083E10E94BB0480930101811119
:100BD000CACF81E40E949104809301018111C3CFA7
:100BE0000E94CC04B82EB094BFCF80E0C0CF0E944A
:100BF000210681E0DF91CF911F910F91FF90EF903F
:100C0000DF90CF90BF900895E82FF0E0ED5BFE4FAE
:100C10008081089508950F931F93CF93DF93C3E4CA
:100C2000D1E010E00C2F025F899190E00E94ED1D51
:100C3000180F0C13F9CF812FDF91CF911F910F91D6
:100C400008950C940F0856985E9825982D9826982C
:100C50002E9827982F988FEF90E09093890080939B
:100C6000880090938B0080938A0090938D008093EE
:100C70008C00259A2D9A2FEF80E792E0215080403A
:100C80009040E1F700C00000269A2E9A2FEF80E7EF
:100C900092E0215080409040E1F700C00000279A88
:100CA0002F9A2FEF80E792E0215080409040E1F7AB
:100CB00000C0000025982D982FEF80E792E021508A
:100CC00080409040E1F700C0000026982E982FEF5A
:100CD00080E792E0215080409040E1F700C00000A2
:100CE00027982F9856985E9825982D9826982E9894
:100CF00027982F98089589EA8093800089E080934F
:100D0000810024982C983F988AB18F748AB96E9884
:100D1000479A8BB1806B8BB9769A0E9423060C940C
:100D20000E0880E2809301018091510181110EC073
:100D30000E948B0481E0809351012FEF83ED90E3BB
:100D4000215080409040E1F700C0000080E40E9404
:100D500091048093010181112EC00E94BB048093F5
:100D60000101811128C00E94BB04809301018111FF
:100D700022C08FE30E94BB048093010181111BC03C
:100D80000E94B30480E40E949104809301018111C8
:100D900012C08CE00E94BB048093010181110BC042
:100DA0000E94BB0480930101811105C08FE30E9462
:100DB000BB04809301010E94B30480910101089556
:100DC000462F50E04031510508F01FC1DC01FA0107
:100DD000EA5AFF4F12968C910C94A9268823A9F009
:100DE0000E94911E90935301809352018091BF0104
:100DF0009091C001A091C101B091C20128E0822769
:100E000088709927AA27BB27AEC08091BF01909117
:100E1000C001A091C101B091C20128E08227887071
:100E20009927AA27BB278093BF019093C001A09365
:100E3000C101B093C20180915201909153010E946F
:100E40009D1E873991050CF0E0C083EA92E0089579
:100E5000882309F4DAC08091BF019091C001A0916C
:100E6000C101B091C20120E2822780729927AA278E
:100E7000BB2779C0882339F00E94911E90935301BB
:100E8000809352010AC080915201909153010E94B7
:100E90009D1E873991050CF4B8C08091BF019091D7
:100EA000C001A091C101B091C20120E182278071EF
:100EB0009927AA27BB2757C0882349F00E94911E73
:100EC00090935301809352018EE992E008958091AE
:100ED0005201909153010E949D1E873991050CF09B
:100EE0008EC080E992E00895882309F48EC08BE7D4
:100EF00092E00895882309F488C086E692E0089578
:100F0000882309F482C081E592E00895882309F4DA
:100F10007CC08CE392E00895882309F476C087E2D0
:100F200092E0089581116EC089E891E008958823C8
:100F300009F46BC080E891E008958823E9F00E94ED
:100F4000911E90935301809352018091BF01909123
:100F5000C001A091C101B091C20124E08227847038
:100F60009927AA27BB278093BF019093C001A09324
:100F7000C101B093C20149C08091520190915301C7
:100F80000E949D1E873991050CF43FC0DECF882357
:100F9000E1F18BE691E008958823B9F186E591E0CF
:100FA0000895882349F00E94911E909353018093E5
:100FB000520181E591E00895809152019091530191
:100FC0000E949D1E873991051CF583E491E00895E8
:100FD000882349F00E94911E9093530180935201FF
:100FE0008CE391E0089580915201909153010E9409
:100FF0009D1E873991057CF48AE291E0089589E984
:1010000092E0089582E292E0089580E090E00895F1
:101010008CE491E0089585E391E00895089560914E
:10102000BF017091C0018091C1019091C2010E94E5
:10103000F91D56985E9825982D9826982E982798F1
:101040002F98823061F018F4813031F008958430A7
:1010500069F0853039F00895259A2D9A0895269AD9
:101060002E9A0895259A2D9A269A2E9A279A2F9A83
:10107000089581E0089581E008950C943B08089557
:101080000F931F93CF93DF938C01FC01C081D1811B
:10109000CE010E94721CBE010E94E908EC01B80159
:1010A0000E943D08882309F48DC0F80182818823BD
:1010B00009F44AC080915F0181111FC0C431F0E57D
:1010C000DF0709F051C00E943F0881E080935F0173
:1010D0000E94911E90935E0180935D0110925601D3
:1010E000109258011092570110925A011092590112
:1010F00010925C0110925B0165C080915D0190913E
:101100005E010E949D1E883C910570F480915601FD
:10111000E82FF0E0EE0FFF1FE95AFE4FD183C083A6
:101120008F5F809356014EC0C43880E5D80721F008
:10113000C538D04501F13AC0F8018281882341F0D9
:101140001092540182E01EC0C438E0E5DE0759F574
:1011500080915401811106C086E20E94FC1386E250
:101160000E94C41482E01CC0C438F0E5DF0741F3DC
:10117000C538D045D9F4F8018281882331F0109226
:10118000550180E20E9413151DC080915501811107
:1011900006C087E20E94FC1387E20E94C41480E22A
:1011A0000E941A150FC0C538D04529F381E08093FD
:1011B000540180935501C801DF91CF911F910F9188
:1011C0000C94390880E0DF91CF911F910F91089521
:1011D000089596E0799FF001112494E5899FE00D30
:1011E000F11D1124E60FF11DEE0FFF1FE455FD4F19
:1011F000859194910895880F991FFC01E45DFE4F3D
:10120000859194910895880F991FFC01E455FD4F35
:101210008591949108950F931F93CF93DF93EC01E1
:10122000811520E3920750F5C11580E2D80708F038
:10123000C3C0CB3BD10590F4C83AD10508F06AC0D1
:10124000C53AD10508F05BC0C430D10508F0D0C163
:10125000219709F0CAC101E010E00AC2CF3FD105D1
:1012600011F008F0C5C1C03FD10508F0A2C0CE0101
:10127000805E9109089708F4BBC1B7C1C13090E501
:10128000D90709F4A2C020F5C0318FE4D80770F463
:10129000C11590E4D90708F094C0C11521E3D20725
:1012A00008F0A3C1DD278E01106CE2C1C115D04545
:1012B00009F09BC10E9479178FEF94E32CE08150D5
:1012C00090402040E1F700C000000E94EC1ED0C119
:1012D000C11597E5D90758F4C03121E5D20708F0C8
:1012E0001CC1C43180E5D80708F475C07EC1CE01A9
:1012F00090578115904108F078C1DF7073C1C53AED
:10130000D10509F477C1C63AD10509F076C102E8E2
:1013100010E4AEC1C83AD10509F472C1C93AD10589
:1013200009F471C1CA3AD10509F470C1CB3AD105AB
:1013300009F46FC1CC3AD10509F46EC1CD3AD1059B
:1013400009F46DC1C03BD10509F46CC1CE3AD10599
:1013500009F46BC1CF3AD10509F46AC1C13BD1058B
:1013600009F469C1C23BD10509F468C1C33BD10589
:1013700009F467C1C43BD10509F466C1C53BD10579
:1013800009F465C1C63BD10509F464C1C73BD10569
:1013900009F463C1C83BD10509F462C1C93BD10559
:1013A00009F461C1CA3BD10509F460C100E014E44D
:1013B0005FC18E0110655CC1CE019F700E94030960
:1013C00058C1DF708E01106A53C18091DC018160C9
:1013D0008093DC014DC10E949120811102C00E94C6
:1013E00077200E94AE2090E09093FD018093FC0155
:1013F000C23080E5D80721F48091FC01816086C06D
:10140000C43090E5D90721F48091FC0182607EC050
:10141000C63020E5D20721F48091FC01846076C0BB
:10142000C83080E5D80719F48091FC0127C0CA3084
:1014300090E5D90721F48091FC01806167C0CC3030
:1014400020E5D20721F48091FC0180625FC0CE309C
:1014500080E5D80721F48091FC01806457C0C03139
:1014600090E5D90721F48091FC0180684FC0C2311A
:1014700020E5D20729F48091FC018460886046C091
:10148000C33080E5D80721F48091FC018E7F3EC0F7
:10149000C53090E5D90721F48091FC018D7F36C0DD
:1014A000C73020E5D20721F48091FC018B7F2EC04C
:1014B000C93080E5D80719F48091FC0126C0CB30F3
:1014C00090E5D90721F48091FC018F7E1FC0CD30BB
:1014D00020E5D20721F48091FC018F7D17C0CF3029
:1014E00080E5D80721F48091FC018F7B0FC0C131CA
:1014F00090E5D90721F48091FC018F7707C0C331B3
:10150000D04531F48091FC018B7F877F8093FC0173
:101510008091FC010E94B220ABC08D2F99278F7063
:10152000992781309105D9F49E012370332702C099
:10153000880F991F2A95E2F79C688E0144E0000FFE
:10154000111F4A95E1F700271370802B912B53E070
:10155000CC0FDD1F5A95E1F7C076DD272FC0823012
:10156000910531F4DC2FCC278E01016F106A80C009
:101570008330910569F4CE018370992701E010E072
:1015800002C0000F111F8A95E2F7C8019C680FC0C6
:1015900084309105B9F4CE018370992701E010E001
:1015A00002C0000F111F8A95E2F7C8019A6823E074
:1015B000CC0FDD1F2A95E1F7C07ED7708C010C2B74
:1015C0001D2B56C08530910531F4DC2FCC278E01C0
:1015D000046F106A4DC0069709F04AC0CF71DD272D
:1015E000DC2FCC278E01106243C000E010E040C029
:1015F0008E013EC001E810E43BC003E810E438C0AF
:1016000002EE14E435C009EE14E432C00AEE14E42C
:101610002FC005EB14E42CC006EB14E429C007EB43
:1016200014E426C00CEC14E423C00DEC14E420C038
:1016300003E815E41DC00AE815E41AC002E915E440
:1016400017C004E915E414C001E216E411C003E276
:1016500016E40EC004E216E40BC005E216E408C06E
:1016600006E216E405C007E216E402C00AE216E448
:10167000C801DF91CF911F910F91089596E0799F56
:10168000F001112494E5899FE00DF11D1124E60F6E
:10169000F11DEE0FFF1FE455FD4F85919491803EA3
:1016A0009105E0F4803C910558F58133910509F4EA
:1016B0006FC048F48932910509F463C08A329105FC
:1016C00009F46DC072C089339105E9F08238910543
:1016D000D1F08533910509F44DC067C0833E910573
:1016E00081F138F4803E9105B9F0823E9105D9F040
:1016F0005CC0863E910561F1873E9105A1F155C020
:101700000E94FB0808952091FC0120FD02C021FFEA
:101710004CC080EE90E049C08091FC0180FFF9CF81
:1017200089E390E042C08091FC0182FF0EC080916D
:10173000FC0184FF03C080E090E037C083EE90E0BE
:1017400034C08091FC0182FFF2CF82EE90E02DC088
:101750008091FC0183FF0BC08091FC0184FDEBCFE5
:1017600087EE90E022C08091FC0183FFF5CF86EEEA
:1017700090E01BC08091FC0185FF07C089E290E0EA
:1017800014C08091FC0185FFF9CF85E390E00DC086
:101790008091FC0186FF07C08AE290E006C080913C
:1017A000FC0186FFF9CF81E390E00E940B090895C8
:1017B00008950C94D80B809170010895CF93DF9316
:1017C00000D01F92CDB7DEB79C018091F301843029
:1017D00019F593E099833B832A839093E9008FEF77
:1017E0009091E800815095FD06C095ED9A95F1F72E
:1017F00000008111F5CF8091E80085FF0DC040E029
:1018000050E063E070E0CE0101960E94480E8091A6
:10181000E8008E778093E8000F900F900F90DF9193
:10182000CF910895CF93DF9300D01F92CDB7DEB74D
:101830002091F301243021F522E029839B838A83C0
:1018400083E08093E9008FEF9091E800815095FD4F
:1018500006C095ED9A95F1F700008111F5CF8091C2
:10186000E80085FF0DC040E050E063E070E0CE018D
:1018700001960E94480E8091E8008E778093E800E0
:101880000F900F900F90DF91CF9108952091F30169
:101890002430F1F422E02093E9002FEF3091E800AA
:1018A000215035FD06C035ED3A95F1F700002111C4
:1018B000F5CF2091E80025FF0BC040E050E065E047
:1018C00070E00E94480E8091E8008E778093E800D7
:1018D0000895CF93DF93EC019091F301943009F0D8
:1018E00046C080910C018823D9F080910D01882396
:1018F000B9F09093E9008FEF9091E800815095FD49
:1019000006C095E19A95F1F700008111F5CF80911D
:10191000E80085FF2CC040E050E060E170E017C0B7
:1019200081E08093E9008FEF9091E800815095FD70
:1019300006C095ED9A95F1F700008111F5CF8091E1
:10194000E80085FF14C040E050E068E070E0CE01A0
:101950000E94480E8091E8008E778093E80080E135
:10196000FE01A0E6B1E001900D928A95E1F7DF91CA
:10197000CF9108958091F201811109C00E94DD0F7D
:101980000E943A108091E20084608093E200089502
:101990001092F201089508950C9421250E94821E50
:1019A0000E9427250E94E0120C94D90B42E061ECC2
:1019B00081E00E94570F42E061EC82E00E94570FE5
:1019C00042E061EC83E00E94570F42E161EC84E069
:1019D0000C94570F8091F501833009F455C030F411
:1019E000813071F0823009F48EC008958A3009F494
:1019F0007AC08B3009F460C0893009F09CC020C0E7
:101A00008091F401813A09F096C08091E800877FC7
:101A10008093E8008091F8019091F901892B21F4DD
:101A200060E180E691E003C060E080E090E070E07B
:101A30000E94930E8091E8008B778093E8000895D0
:101A40008091F401813209F076C08091F801909183
:101A5000F901009719F0039709F06DC08091E80033
:101A6000877F8093E8008091E80082FD05C0809127
:101A7000F3018111F8CF5FC08091F1008093700174
:101A80008091E8008B7753C08091F401813A09F08E
:101A900052C08091F8019091F901892B09F04BC057
:101AA0008091E800877F8093E8008091E80080FFC4
:101AB000FCCF80910C0136C08091F4018132D9F5C0
:101AC0008091F8019091F901892BA9F58091E800A6
:101AD000877F8093E8000E948C0F8091F6018093AD
:101AE0000C010C9479178091F401813221F58091D9
:101AF000E800877F8093E8000E948C0F8091F701B7
:101B00008093710108958091F401813AA1F480914C
:101B1000E800877F8093E8008091E80080FFFCCF99
:101B2000809171018093F1008091E8008E7780931D
:101B3000E8000C948C0F089584B7877F84BF88E1F8
:101B40000FB6F89480936000109260000FBE90E092
:101B500080E80FB6F89480936100909361000FBE07
:101B60000E942F130E94DD0F0E943A108091E20024
:101B700084608093E20078940E94C0120E94311326
:101B800082E091E00E94DB120E940F258091F30118
:101B9000853069F40E94491E8091F1018823B1F3D8
:101BA0000E94741E882391F30E94320EEFCF0E9490
:101BB0003713ECCF292F332723303105C9F064F4D4
:101BC0002130310581F02230310509F043C08DE626
:101BD00090E020ED36E042C021323105F1F02232B2
:101BE000310541F137C082E190E02DE337E036C0A6
:101BF00099278130910541F08230910541F0892B80
:101C000049F5ECECF6E005C0E4EBF6E002C0ECE9E7
:101C1000F6E0849190E09F0121C06430D8F4E62F73
:101C2000F0E0EE0FFF1FEE5DFE4F2081318189E075
:101C300090E014C0643070F470E0FB01EE0FFF1F01
:101C4000E65EFE4F20813181FB01EA5EFE4F80811E
:101C500090E004C080E090E020E030E0FA013183C1
:101C60002083089580E189BD82E189BD09B400FE29
:101C7000FDCF8091D8008F7D8093D8008091E000C7
:101C800082608093E0008091E00081FDFCCF0895A8
:101C9000CF92DF92EF92FF920F931F93CF93DF9338
:101CA000EC018B016A010E94AB0F811133C0C1149A
:101CB000D10439F0F60180819181081B190BC80FFE
:101CC000D91FE12CF12C0115110519F18091E800C3
:101CD00085FD16C08091E8008E778093E800C114DE
:101CE000D10449F0F60180819181E80EF91EF1825C
:101CF000E08285E00FC00E94AB0F882321F30AC069
:101D000089918093F10001501109FFEFEF1AFF0A4A
:101D1000DACF80E0DF91CF911F910F91FF90EF908C
:101D2000DF90CF9008952091FA013091FB012617A2
:101D3000370748F06115710539F42091E8002E77D6
:101D40002093E80001C0B90140E061157105A9F1D7
:101D50002091F301222309F443C0253009F442C045
:101D60002091E80023FD40C02091E80022FD32C010
:101D70002091E80020FFE9CF4091F3002091F2008C
:101D800030E0342BFC01CF016115710559F028308A
:101D9000310540F481918093F100615071092F5F0A
:101DA0003F4FF1CF41E02830310509F040E020916C
:101DB000E8002E772093E800C8CF4111C9CF0AC0B0
:101DC0008091F301882361F0853061F08091E80013
:101DD00083FD0AC08091E80082FFF2CF80E0089581
:101DE00082E0089583E0089581E008952091FA014A
:101DF0003091FB012617370748F06115710539F45A
:101E00002091E8002E772093E80001C0B901FC0181
:101E100020E06115710591F18091F301882309F4A7
:101E200040C0853009F43FC08091E80083FD3DC08B
:101E30008091E80082FD2FC08091E80080FFE9CF0B
:101E40002091F3008091F20090E0922B61157105D2
:101E500059F08830910540F424912093F100319697
:101E6000615071090196F2CF21E0089709F020E056
:101E70008091E8008E778093E800CBCF2111CCCF02
:101E80000AC08091F301882361F0853061F0809170
:101E9000E80083FD0AC08091E80082FFF2CF80E075
:101EA000089582E0089583E0089581E00895982FD1
:101EB000973058F59093E900981739F07091EC003D
:101EC0002091ED005091F00003C0242F762F50E0B8
:101ED00021FF19C03091EB003E7F3093EB00309131
:101EE000ED003D7F3093ED003091EB003160309399
:101EF000EB007093EC002093ED005093F0002091E4
:101F0000EE0027FF07C09F5FD3CF8F708093E9005B
:101F100081E0089580E008958091F40187FF11C069
:101F20008091E80082FD05C08091F3018111F8CF16
:101F300011C08091E8008B770BC08091F30188235A
:101F400049F08091E80080FFF8CF8091E8008E771B
:101F50008093E80008952091E4003091E50095E633
:101F60004091EC00842F817040FF22C08091E800F6
:101F700080FD1CC08091F301882391F0853091F0A1
:101F80008091EB0085FD10C04091E4005091E50088
:101F90004217530729F39A01915011F784E00895ED
:101FA00082E0089583E0089581E0089580E0089537
:101FB0004091E80042FFDECF08950E944B100E943E
:101FC0005310E0EEF0E0808181608083E8EDF0E086
:101FD00080818F77808319BCA7EDB0E08C918E7FD4
:101FE0008C9380818F7E80831092F20108950F93ED
:101FF0001F93CF93DF930E944B100E945310C8EDA4
:10200000D0E088818F778883888180688883888101
:102010008F7D888319BC1092F3011092EF0110920A
:10202000F1011092F00100EE10E0F80180818B7F49
:10203000808388818160888342E060E080E00E9444
:10204000570FE1EEF0E080818E7F8083E2EEF0E0DA
:10205000808181608083808188608083F8018081B5
:102060008E7F8083888180618883DF91CF911F91EB
:102070000F910895E8EDF0E080818F7E8083E7ED99
:10208000F0E080818160808384E082BF81E0809382
:10209000F2010C94F70FE8EDF0E080818E7F8083F1
:1020A0001092E20008951092DA001092E100089573
:1020B0001F920F920FB60F9211242F933F934F93BD
:1020C0005F936F937F938F939F93AF93BF93EF93A0
:1020D000FF938091E10082FF0BC08091E20082FFBC
:1020E00007C08091E1008B7F8093E1000E94BF12C6
:1020F0008091DA0080FF1FC08091D80080FF1BC054
:102100008091DA008E7F8093DA008091D90080FF81
:102110000DC080E189BD82E189BD09B400FEFDCF1B
:1021200081E08093F3010E94BA0C05C019BC1092A3
:10213000F3010E94C80C8091E10080FF19C08091DA
:10214000E20080FF15C08091E2008E7F8093E20064
:102150008091E20080618093E2008091D8008062EB
:102160008093D80019BC85E08093F3010E94CC0CC9
:102170008091E10084FF30C08091E20084FF2CC098
:1021800080E189BD82E189BD09B400FEFDCF809167
:10219000D8008F7D8093D8008091E1008F7E80935E
:1021A000E1008091E2008F7E8093E2008091E20066
:1021B00081608093E2008091EF01882311F084E038
:1021C00007C08091E30087FD02C081E001C083E089
:1021D0008093F3010E94CE0C8091E10083FF29C01F
:1021E0008091E20083FF25C08091E100877F80938A
:1021F000E10082E08093F3011092EF018091E10011
:102200008E7F8093E1008091E2008E7F8093E200D8
:102210008091E20080618093E20042E060E080E033
:102220000E94570F8091F00088608093F0000E9418
:10223000CB0CFF91EF91BF91AF919F918F917F91C7
:102240006F915F914F913F912F910F900FBE0F9023
:102250001F9018951F920F920FB60F9211242F9373
:102260003F934F935F936F937F938F939F93AF931E
:10227000BF93CF93DF93EF93FF93C091E900CF70AB
:102280008091EC00D82FD17080FDD0E81092E90049
:102290008091F000877F8093F00078940E946E1107
:1022A0001092E9008091F00088608093F000CD2BBF
:1022B000CF70C093E900FF91EF91DF91CF91BF9173
:1022C000AF919F918F917F916F915F914F913F91CE
:1022D0002F910F900FBE0F901F9018951F93CF93C3
:1022E000DF93CDB7DEB7AA970FB6F894DEBF0FBE67
:1022F000CDBFE4EFF1E088E08E0F9091F100919373
:102300008E13FBCF0E94EA0C8091E80083FF1FC16F
:102310008091F4019091F501492F50E04A30510528
:1023200008F015C1FA01EA59FF4F0C94A92680382C
:1023300081F0823809F00BC18091F8018F70809391
:10234000E9008091EB0085FB882780F91092E90075
:1023500006C08091F0019091F101911182609091FD
:10236000E800977F9093E8008093F1001092F100CD
:10237000C8C0282F2D7F09F0EAC0882319F08230C9
:1023800061F0E5C08091F601813009F0E0C0933042
:1023900009F080E08093F1012BC08091F60181115A
:1023A00027C08091F8018F7009F4D1C08093E900B3
:1023B0002091EB0020FF1CC0933021F48091EB00B2
:1023C000806214C09091EB0090619093EB0021E04B
:1023D00030E0A90102C0440F551F8A95E2F74093EF
:1023E000EA001092EA008091EB0088608093EB0095
:1023F0001092E9008091E800877F86C08111A7C014
:102400001091F6011F778091E3008078812B8093F3
:10241000E3008091E800877F8093E8000E948C0FA2
:102420008091E80080FFFCCF8091E300806880937A
:10243000E300111102C082E001C083E08093F30148
:1024400086C08058823008F082C08091F601909159
:10245000F7018C3D53E0950779F583E08A838AE2A2
:1024600089834FB7F894DE01139620E03EE051E2F5
:10247000E32FF0E050935700E49120FF03C0E29572
:10248000EF703F5FEF708E2F90E0EA3010F0C7964C
:1024900001C0C0968D939D932F5F243149F74FBFA4
:1024A0008091E800877F8093E8006AE270E0CE01C7
:1024B00001960E94930E14C0AE014F5F5F4F609172
:1024C000F8010E94DA0DBC01009709F440C0909118
:1024D000E800977F9093E80089819A810E94F60E28
:1024E0008091E8008B778093E80031C0803879F5DF
:1024F0008091E800877F8093E8008091EF018093CE
:10250000F1008091E8008E778093E8000E948C0FA4
:102510001EC081111CC09091F6019230C0F48091D0
:10252000E800877F8093E8009093EF010E948C0F72
:102530008091EF01811106C08091E30087FD02C008
:1025400081E001C084E08093F3010E94D60C809169
:10255000E80083FF0AC08091E800877F8093E8004D
:102560008091EB0080628093EB00AA960FB6F894FE
:10257000DEBF0FBECDBFDF91CF911F9108950895AB
:10258000CF938091F3018823A1F0C091E900CF702F
:102590009091EC00892F817090FD80E8C82B1092FB
:1025A000E9008091E80083FD0E946E11CF70C09316
:1025B000E900CF9108959093770180937601089573
:1025C000E0917601F0917701309721F00190F08150
:1025D000E02D099480E00895E0917601F091770173
:1025E000309721F00280F381E02D09940895E09165
:1025F0007601F0917701309721F00480F581E02D8C
:102600000994089520917401309175018217930700
:1026100071F09093750180937401E0917601F091CF
:102620007701309721F00680F781E02D0994089515
:1026300020917201309173018217930771F090938A
:10264000730180937201E0917601F09177013097E8
:1026500021F00084F185E02D0994089508950C94EB
:102660002E130E94881E0E94FE040C944A1F9F9203
:10267000AF92BF92CF92DF92EF92FF920F931F9390
:10268000CF93DF9300D000D000D0CDB7DEB70E944B
:1026900016050DE010E0AA24A394B12C902E802FF3
:1026A0000E940406980127583E4F6901F901F08005
:1026B000F826A1F40150110988F78FEF89838A83E6
:1026C0001B820E94911E8160782F9D838C8349819B
:1026D0005A816B818D810E94CE132FC09091DC01B5
:1026E00091FF04C08E830E940A068E8125E030E0AF
:1026F000A501022E01C0440F0A94EAF7E42E4F21EF
:10270000C1F029839A828E2191E009F490E09B83A5
:102710000E94911E8160782F9D838C8349815A810C
:102720006B818D810E94CE13F6018081E826E082C4
:1027300004C021503109E0F6BDCF0E943122109132
:1027400078010E94E0121817B9F00E94E0128093FD
:10275000780126960FB6F894DEBF0FBECDBFDF918D
:10276000CF911F910F91FF90EF90DF90CF90BF908E
:10277000AF909F900C94D90B26960FB6F894DEBFBD
:102780000FBECDBFDF91CF911F910F91FF90EF90C2
:10279000DF90CF90BF90AF909F900895CF93DF933D
:1027A000CDB7DEB72B970FB6F894DEBF0FBECDBF07
:1027B0004F83588769877A878B87DE01119686E079
:1027C000FD0111928A95E9F785E0FE0137960190A7
:1027D0000D928A95E1F749815A816B817C818D81C7
:1027E0009E810E94171A2B960FB6F894DEBF0FBE7B
:1027F000CDBFDF91CF910895CF93882309F4C2C054
:10280000C82F823859F40E94E01281FDBBC089E3D1
:102810000E94F11C0E94BE1D89E30CC0833879F42C
:102820000E94E01280FDAEC083E50E94F11C0E9470
:10283000BE1D83E50E94331DCF910C94BE1D8438CC
:1028400059F40E94E01282FD9DC087E40E94F11CB1
:102850000E94BE1D87E4EECF8CEF8C0F813A48F4C6
:102860008C2F0E94742481118DC08C2F0E94F11C2A
:10287000E3CF80E28C0F883048F4C77081E001C05C
:10288000880FCA95EAF70E94771DD6CF8BE58C0F8B
:10289000833078F4C53A29F0C63A31F083E890E005
:1028A00005C081E890E002C082E890E0CF910C94EE
:1028B000021388E58C0F833108F064C0C83A39F1FF
:1028C000C93A41F1CA3A49F1CB3A51F1CC3A59F1FE
:1028D000CD3A61F1C03B69F1CE3A71F1CF3A79F16D
:1028E000C13B81F1C23B89F1C33B91F1C43B99F1FA
:1028F000C53BA1F1C63BA9F1C73BB1F1C83BB9F15A
:10290000C93BC1F1CA3BC9F180E090E038C082EE1A
:1029100090E035C089EE90E032C08AEE90E02FC0A2
:1029200085EB90E02CC086EB90E029C087EB90E02F
:1029300026C08CEC90E023C08DEC90E020C083E8B2
:1029400091E01DC08AE891E01AC082E991E017C0C9
:1029500084E991E014C081E292E011C083E292E048
:102960000EC084E292E00BC085E292E008C086E2ED
:1029700092E005C087E292E002C08AE292E0CF9145
:102980000C941813CF910895882309F44BC0823812
:1029900059F40E94E01281FF45C089E30E94F11CB6
:1029A0000E94BE1D89E30CC0833871F40E94E012BE
:1029B00080FF38C083E50E94F11C0E94BE1D83E5A4
:1029C0000E94331D0C94BE1D843859F40E94E012FD
:1029D00082FF28C087E40E94F11C0E94BE1D87E48C
:1029E000EFCF9CEF980F913A58F390E2980F983000
:1029F00050F4877091E001C0990F8A95EAF7892F0A
:102A00000E947D1DDFCF9BE5980F933020F480E07E
:102A100090E00C940213885A833120F480E090E017
:102A20000C9418130895882321F00E94771D0C94AC
:102A3000BE1D0895882321F00E947D1D0C94BE1DAB
:102A400008957F928F929F92AF92BF92CF92DF9222
:102A5000EF92FF920F931F93CF93DF931F92CDB707
:102A6000DEB77C01C62E772EFC01058102950F7022
:102A7000128111110E94941D0E94EA1C882379F092
:102A8000112369F080E28C0D883048F082E00E94CA
:102A9000D31C0E94EA1C91E0D82ED92601C0D12C6B
:102AA000E72DE295EF70F0E0E059FF4F0C94A92676
:102AB000872D807F072D0F70882311F00295007FEE
:102AC000112389F0002309F490C180E28C0D883035
:102AD00020F4802F0E94771D03C0802F0E94871D45
:102AE0000E94BE1D82C18C2D0E94C414002309F4D3
:102AF00095C180E28C0D883020F4802F0E947D1DCE
:102B000003C0802F0E948D1D0E94BE1D87C1972D7E
:102B1000907F872D8F70903211F08295807FCC202E
:102B200021F0F1E0CF16B1F01EC0112349F00023CF
:102B300009F414C1013009F011C10E94A71D6EC132
:102B4000002319F0013009F469C189830E94AA1D8C
:102B500089810AC1112321F0023008F05FC1FEC053
:102B600001115CC101C1112321F0002309F4F6C059
:102B70003CC1002309F4F8C03EC1872D8695869597
:102B8000837090E0009719F0019761F047C111231D
:102B900021F08C2D972D937002C080E090E00E9470
:102BA00002133CC1112321F08C2D972D937002C08C
:102BB00080E090E00E94181331C18C2D112319F090
:102BC0000E94392102C00E94A1210E94262226C112
:102BD000872D837009F052C0111120C18C2D829570
:102BE00086958770880F880F9C2D9F70892E912C59
:102BF000A12CB12C082E04C0880C991CAA1CBB1C4B
:102C00000A94D2F7C4FE14C00FE010E020E030E0D8
:102C1000B901A80104C0440F551F661F771F8A958C
:102C2000D2F7CB01BA01609570958095909503C05D
:102C300060E070E0CB01272D26952695237030E0CB
:102C40002230310569F02330310589F0682979296E
:102C50008A299B292130310571F00E945F1BDEC05B
:102C6000682979298A299B290E947B1BD7C00E9449
:102C70005F1BC501B4010E94431BD0C0112319F092
:102C8000872D817001C08695882309F4C7C08C2DDB
:102C9000829586958770880F880F9C2D9F70892E4E
:102CA000912CA12CB12C082E04C0880C991CAA1CB4
:102CB000BB1C0A94D2F7C4FE14C00FE010E020E061
:102CC00030E0B901A80104C0440F551F661F771FEB
:102CD0008A95D2F7CB01BA01609570958095909551
:102CE00003C060E070E0CB01272D26952695237068
:102CF000422F50E04230510569F04330510589F0D0
:102D0000682979298A299B294130510571F00E944F
:102D1000391C84C0682979298A299B290E94551C5D
:102D20007DC00E94391CC501B4010E941D1C76C0E3
:102D30008C2D90E0FC01E05EF109E531F10508F031
:102D400050C0E058FF4F0C94A9260C2D0F70872D12
:102D50008F71112331F00E94B61B802F0E94131532
:102D60005DC00E94D71B802F0E941A1557C01123E7
:102D700039F0011153C0872D8F710E94FC1B4EC08A
:102D8000023008F04BC0F7CF112339F0872D8F7137
:102D90000E94B61B43C01123C9F3872D8F710E9477
:102DA000D71B3CC0112329F0872D8F710E94A11BD6
:102DB00035C00E94971B32C0112351F0172D1F718F
:102DC000812F0E94B61B63E0812F0E94CA1C26C07F
:102DD00081E00E94D31C023008F182E00E94D31CE3
:102DE0001DC0112331F0002389F28C2D0E94FC13A9
:102DF00015C0002391F28C2D0E94C4140FC0472DE2
:102E00004F706C2DC7010E94E0060E94BB1A06C0DD
:102E1000472D4F706C2DC7010E94E808DD20F9F0A6
:102E20000E94C61C80FD1BC0F70112820E94C01CBC
:102E30000E94B61BC7010E943E170E94C01C0F9043
:102E4000DF91CF911F910F91FF90EF90DF90CF9086
:102E5000BF90AF909F908F907F900C94D71B0F9056
:102E6000DF91CF911F910F91FF90EF90DF90CF9066
:102E7000BF90AF909F908F907F9008950F931F9376
:102E8000CF93DF93EC01888199812B813C81232BA7
:102E9000B9F09F3F11F48F3F99F0CE010E94400896
:102EA000882371F0688179818A810E94BC1C8C0121
:102EB0000E94711C0E94381BB801CE010E9421158E
:102EC000DF91CF911F910F9108950E94941D0E9450
:102ED000A41D0E94691D0E94BE1D0E94D7220E944F
:102EE000262280E090E00E94021380E090E00C94A3
:102EF00018130E94841D0C9465170E94B11C292F81
:102F000022952F7030E02C3031054CF42A303105F9
:102F10006CF42250310922303105A8F407C02C305E
:102F2000310569F02F30310551F00DC0803F69F057
:102F300018F4803E40F409C0843F29F406C093FB96
:102F4000882780F9089580E0089581E00895CF935F
:102F5000DF9300D000D01F92CDB7DEB70F900F9057
:102F60000F900F900F90DF91CF910895CF93DF9343
:102F700000D000D000D0CDB7DEB726960FB6F894BB
:102F8000DEBF0FBECDBFDF91CF9108951F93CF93CA
:102F9000DF93C091870116E080918801C81799F0EE
:102FA000D0E01C9FF0011D9FF00D1124E757FE4F4C
:102FB0004081518162817381848195810E94B6171D
:102FC0002196C770E9CFDF91CF911F91089540916D
:102FD000B9015091BA016091BB017091BC0180911F
:102FE000BD019091BE010C94B6178091BE018295EF
:102FF0008F7009F054C08091BB01882309F44FC041
:1030000080918701A09188016091B9017091BA0106
:103010004091BC015091BD01B6E08A1709F43FC050
:1030200090E041155105C1F17F3F11F46F3FA1F1CF
:10303000B89FF001B99FF00D1124E757FE4F218191
:1030400072132AC02081621327C02281211124C05B
:10305000238134812417350710F421503109241BB2
:10306000350B283C3105C0F42091BE012F70206142
:103070002093BE0126E0289FF001299FF00D112426
:10308000E257FE4F80818F708061808389EB91E0F1
:103090000E943E170C94C61701968770BECF089504
:1030A000CF92DF92EF92FF920F931F93CF93DF9314
:1030B000CDB7DEB762970FB6F894DEBF0FBECDBFB7
:1030C0008C0185E0F801DE011D9601900D928A9534
:1030D000E1F7D8014C9111965C91119712966C9181
:1030E00012971396CD90DC9014973091B90170919E
:1030F000BA018091BC019091BD01009709F46BC1A8
:103100007F3F19F43F3F09F466C1E090BB01EE2018
:1031100009F4C0C02091BE01C816D90628F0F601F6
:10312000E81BF90BCF0104C0809590958C0D9D1D77
:10313000FF24F394883C910578F0F12C207F09F06E
:10314000C6C07C2DD98AC88A89890E94A71789EBB5
:1031500091E00E943E17B1C0822F807F09F046C0E7
:10316000751314C0341312C0611110C02F70206188
:103170002093BE010E94E71789EB91E00E943E1761
:103180008091BE01D80115968C932EC0CD2819F1DF
:103190005F3F11F44F3FF9F0F62E61111CC0809192
:1031A00087012091880136E0821709F45AC090E027
:1031B000389FF001399FF00D1124E757FE4F7181C0
:1031C000571306C07081471303C07281711103C089
:1031D00001968770E9CFF62E662309F418C1809115
:1031E000BE0181608093BE01F12C11C1751308C02E
:1031F000341306C0611104C08091BE01D801C3C060
:103200004D875E878D859E856A8B0E947D176A89B2
:103210008823E1F16623D1F12091BE01822F8295AE
:103220008F7090E0029774F08091B9019091BA018B
:1032300098878F831986DB86CA862C87CE010796EE
:103240000E943E1786E0F801A9EBB1E001900D92D3
:103250008A95E1F70E94F5170E94E717FF24F3947F
:10326000D6C04D875E878D859E850E94B11C292F13
:1032700022952F7030E0223031050CF0BCC09F70D9
:1032800009F0B6C0805E883008F4C1C0C8010E9451
:103290003E17E4CFC816D90608F453C0F601E81B60
:1032A000F90BCF01883C910508F450C0F12C7C2D1E
:1032B000D98AC88A89890E94A717E9EBF1E086E0DC
:1032C000DF011D928A95E9F70E94E717A0C07513E8
:1032D00014C0341312C0611110C08091BE01F801F6
:1032E0008583C8010E943E1786E0E9EBF1E0DF012B
:1032F0001D928A95E9F7FE2C8AC04D875E878D85E1
:103300009E856A8B0E947D176A89882309F4BECF47
:10331000662309F4BBCF2091BE01822F82958F7066
:1033200090E002970CF48ECF8091B9019091BA0190
:103330009A8389831B82DD82CC822E83CE01019603
:103340007FCF809590958C0D9D1DACCFF62E66237A
:1033500009F49CCF75132EC034132CC02091BE01EC
:1033600020FD1FC0822F82958F70D9F0D80115964D
:103370002C9315978F3049F08F5F982F9295907FFF
:10338000822F8F70892B15968C93C8010E943E174F
:1033900086E0F801A9EBB1E001900D928A95E1F782
:1033A00093CF86E0F801A9EBB1E001900D928A95E8
:1033B000E1F72DC04D875E878D859E850E947D1724
:1033C000811140CF8091BE0181608093BE01C80110
:1033D0000E943E171CC0662309F458CF4D875E87B4
:1033E0008D859E850E947D17882309F44FCF2ACFB3
:1033F000811148CF0CC0243031050CF047CF9F70AD
:1034000009F440CFF8019581907F09F03BCF8F2DD3
:1034100062960FB6F894DEBF0FBECDBFDF91CF919D
:103420001F910F91FF90EF90DF90CF9008951F9321
:10343000CF93DF93CDB7DEB72C970FB6F894DEBFEE
:103440000FBECDBF4F83588769877A878B879C874C
:10345000CE0107960E945018882369F08F819885C5
:103460002A853B85232BF1F19F3F09F063C08F3FF5
:1034700009F060C037C086E0FE013796DE01119684
:1034800001900D928A95E1F76F817885EA85FB8539
:10349000309741F17F3F11F46F3F21F12091880176
:1034A00030E0C9010196877099274091870150E06B
:1034B0008417950709F447C069837A83FD83EC83F9
:1034C00096E0929FD001939FB00D1124A757BE4F55
:1034D000FE01319601900D929A95E1F78093880153
:1034E0000E94C61716E08091870190918801891784
:1034F000C1F1189FC001112487579E4F0E94501898
:10350000882379F1E09187011E9FF0011124E7578C
:10351000FE4F4081518162817381848195810E9437
:10352000B6178091870190E0019687709927809364
:103530008701D9CF4F81588569857A858B859C8590
:103540000E94B617CFCF0E9479171092880110926F
:103550008701E9EBF1E086E0DF011D928A95E9F74A
:10356000C1CF2C960FB6F894DEBF0FBECDBFDF9152
:10357000CF911F910895EF92FF920F931F93CF93D6
:10358000DF938C01009709F46CC0F12CEE24E394D6
:10359000E8012196F8018491843740F4843008F0E2
:1035A00051C0813081F0823019F15BC0853709F458
:1035B00044C0A8F19CE7980F903708F052C08F776D
:1035C0000E94C41441C00E5F1F4FFE01C49180E2EF
:1035D0008C0F883048F4C7708E2D01C0880FCA95B3
:1035E000EAF70E94971D14C08C2F0E94FC132DC077
:1035F0000E5F1F4FFE01C49180E28C0F883058F49B
:10360000C7708E2D01C0880FCA95EAF70E949D1DD4
:103610000E94BE1D1AC08C2F0E94C41416C00E5FDB
:103620001F4FFE01C491CC2381F08FE99FE00197E9
:10363000F1F700C00000C150F6CF0E5F1F4FFE0132
:10364000F49003C00E94FC138E018F2D882309F48F
:103650009FCFEFE9FFE03197F1F700C00000815004
:10366000F5CFDF91CF911F910F91FF90EF900895CB
:1036700008956093C3017093C4018093C501909332
:10368000C6010C9465170F931F930091C30110910D
:10369000C4012091C5013091C601DC01CB01802B12
:1036A000912BA22BB32B8093C3019093C401A093C1
:1036B000C501B093C6011F910F910C9465170F932C
:1036C0001F930091C3011091C4012091C501309155
:1036D000C601DC01CB0180239123A223B323809375
:1036E000C3019093C401A093C501B093C6011F917B
:1036F0000F910C9465170F931F930091C3011091C4
:10370000C4012091C5013091C601DC01CB018027A5
:103710009127A227B3278093C3019093C401A0935C
:10372000C501B093C6011F910F910C9465171092BB
:10373000BF011092C0011092C1011092C2010C94FD
:10374000651741E050E060E070E004C0440F551F91
:10375000661F771F8A95D2F74093BF015093C0012F
:103760006093C1017093C2010C94651741E050E071
:1037700060E070E004C0440F551F661F771F8A95F4
:10378000D2F78091BF019091C001A091C101B09189
:10379000C201482B592B6A2B7B2B4093BF015093BE
:1037A000C0016093C1017093C2010C94651741E0A0
:1037B00050E060E070E004C0440F551F661F771FA3
:1037C0008A95D2F740955095609570958091BF018C
:1037D0009091C001A091C101B091C2014823592329
:1037E0006A237B234093BF015093C0016093C101C2
:1037F0007093C2010C94651741E050E060E070E006
:1038000004C0440F551F661F771F8A95D2F7809119
:10381000BF019091C001A091C101B091C2014827A0
:1038200059276A277B274093BF015093C0016093BB
:10383000C1017093C2010C9465170F931F930091FF
:10384000BF011091C0012091C1013091C201DC0182
:10385000CB01802B912BA22BB32B8093BF01909394
:10386000C001A093C101B093C2011F910F910C94AC
:1038700065170F931F930091BF011091C001209114
:10388000C1013091C201DC01CB0180239123A2232D
:10389000B3238093BF019093C001A093C101B09363
:1038A000C2011F910F910C9465170F931F93009104
:1038B000BF011091C0012091C1013091C201DC0112
:1038C000CB0180279127A227B3278093BF01909334
:1038D000C001A093C101B093C2011F910F910C943C
:1038E00065170895CF92DF92EF92FF920F931F9387
:1038F000CF93DF938C01C090C301D090C401E090BE
:10390000C501F090C6018091BF019091C001A091C6
:10391000C101B091C201C82AD92AEA2AFB2ACFE103
:10392000D0E0D701C6010C2E04C0B695A795979597
:1039300087950A94D2F780FF06C0B8018C2F0E94A9
:103940003E0B019721F4219760F780E001C08C2F96
:10395000DF91CF911F910F91FF90EF90DF90CF906B
:103960000895CF93DF93EC010E94721CBE010E9468
:103970003E0BDF91CF910895CB010E94B11C0895B9
:103980008091C70185958595859508958091C7019A
:103990008770089598E0899F90011124262B209329
:1039A000C7010C94B61B2091C70180958223809398
:1039B000C701982F977069F430E0482F552747FDCD
:1039C00050952417350729F08595859585950C9494
:1039D000D71B08959091C701977081E009F480E0AA
:1039E000089590910C01992321F090910D0191116E
:1039F00009C020910E0130910F01F90132969FEF1D
:103A000040E01FC0982F9695969596959F3050F55B
:103A1000E0910E01F0910F01E90FF11D877021E097
:103A200030E0A90102C0440F551F8A95E2F7CA0190
:103A30009181892B818308959F3F39F04F5F4E30EC
:103A400041F051915813F8CF0DC05111F7CF942F79
:103A5000F5CF9F3F39F0F901E90FF11D97FDFA9578
:103A600082830895089590910C01992321F09091FB
:103A70000D01911109C020910E0130910F01F90142
:103A80003296205F3F4F1FC0982F9695969596953A
:103A90009F30F0F4E0910E01F0910F01E90FF11D5C
:103AA000877021E030E0A90102C0440F551F8A95BC
:103AB000E2F7CA0180959181892381830895319627
:103AC000E217F30729F090819813F9CF1082F7CF0E
:103AD000089581E090E0E0910E01F0910F01E80F70
:103AE000F91F1082019680319105A9F708959091F0
:103AF000DB01892B8093DB01089580959091DB0198
:103B000089238093DB0108951092DB010895909141
:103B1000DA01892B8093DA01089580959091DA017A
:103B200089238093DA0108951092DA010895909123
:103B3000D901892B8093D901089580959091D9015D
:103B400089238093D90108951092D9010895809313
:103B5000C80108951092C801089580910E019091B6
:103B60000F01FC0131969C01205F3F4F80E0919155
:103B700091118F5FE217F307D1F70895E0910E01DD
:103B8000F0910F018091DB018083E0910E01F091B3
:103B90000F0190818091DA01892B8083E0910E01E1
:103BA000F0910F0190818091D901892B80838091C0
:103BB000C801882361F0E0910E01F0910F0190811E
:103BC000892B80830E94AD1D81111092C8018091C4
:103BD0000E0190910F010C94EC1220E0009739F047
:103BE000AC0141505109842395232F5FF7CF822FD9
:103BF0000895CF92DF92EF92FF926C01EE24FF24A2
:103C0000C114D104E104F10421F0C701B60120E19F
:103C100001C020E0C72ED82EE92EFF24C114D10404
:103C2000E104F10419F0285FC701B6016B017C01C2
:103C300054E0F694E794D794C7945A95D1F7C114F9
:103C4000D104E104F10419F02C5FC701B6016B0146
:103C50007C0142E0F694E794D794C7944A95D1F753
:103C6000C114D104E104F10419F02E5FC701B601BB
:103C7000DC01CB01B695A79597958795892B8A2B63
:103C80008B2B09F02F5F822FFF90EF90DF90CF906A
:103C900008958091F301843021F11092DD0120E438
:103CA00088E190E00FB6F894A895809360000FBE6D
:103CB0002093600080E00E94D90B83B7817F8460ED
:103CC00083BF83B7816083BF7894889583B78E7FE5
:103CD00083BF88E10FB6F894809360001092600073
:103CE0000FBE0895089508950E94721E0E94160541
:103CF0000E94731E0E940B0691E0811101C090E0AA
:103D0000892F08950E9479170E94E0120C94D90B14
:103D100082E084BD93E095BD9AEF97BD80936E00DD
:103D200008952FB7F8948091DE019091DF01A09162
:103D3000E001B091E1012FBF0895CF92DF92EF92A1
:103D4000FF920F931F932FB7F8944091DE0150918B
:103D5000DF016091E0017091E1012FBF6A017B01F9
:103D6000EE24FF248C0120E030E0C016D106E206EC
:103D7000F30610F4415051099A01281B390BC9016F
:103D80001F910F91FF90EF90DF90CF9008951F92B9
:103D90000F920FB60F9211248F939F93AF93BF93FF
:103DA0008091DE019091DF01A091E001B091E101ED
:103DB0000196A11DB11D8093DE019093DF01A093B8
:103DC000E001B093E101BF91AF919F918F910F906E
:103DD0000FBE0F901F9018950E94DD0FF8942FEFE3
:103DE00087EA91E6215080409040E1F700C0000052
:103DF00087E090EBDC018093FD019093FE01A0939E
:103E0000FF01B09300029CE088E10FB6F894A895FA
:103E1000809360000FBE90936000FFCFEF92FF92FF
:103E20000F931F93CF93DF93D82FCDE08C2F0E9459
:103E3000040605E010E0E82EF12CC701002E02C0B8
:103E4000959587950A94E2F780FF09C0602F7C2F33
:103E500080E00E94E908D81302C081E006C001504A
:103E6000110958F7C15010F780E0DF91CF911F91F1
:103E70000F91FF90EF900895CF93C82F8CE20E948E
:103E80000E1F882321F08C2FCF910C940E1F80E001
:103E9000CF910895CF930E949120811102C00E947A
:103EA0007720C5E6C15049F00E9416058FE39CE9D2
:103EB0000197F1F700C00000F5CF89E20E943C1F96
:103EC000811113C18AE20E943C1F81110E94772058
:103ED00085E00E943C1F81110E94EC1E0E949C20E4
:103EE0008093DC0187E00E943C1F8823A9F18BE1CD
:103EF0000E943C1F882351F08091DC0181FB222726
:103F000020F991E0922790FB81F90EC08EE00E948B
:103F10003C1F882361F08091DC0182FB222720F97D
:103F200091E0922790FB82F98093DC0115C080E13B
:103F30000E943C1F9091DC01882341F093FB2227D3
:103F400020F981E0822780FB93F904C0892F8095B6
:103F500080FB90F99093DC018091DC010E94A0200D
:103F60000E94AE208093FC0180EE0E943C1F8823BB
:103F700041F08091FC01982F909590FB80F98093FF
:103F8000FC0189E30E943C1F882359F08091FC01C9
:103F900081FB222720F991E0922790FB81F9809301
:103FA000FC0182EE0E943C1F882359F08091FC01A5
:103FB00082FB222720F991E0922790FB82F98093DF
:103FC000FC0186EE0E943C1F882359F08091FC0181
:103FD00083FB222720F991E0922790FB83F98093BD
:103FE000FC0183EE0E943C1F882359F08091FC0164
:103FF00084FB222720F991E0922790FB84F980939B
:10400000FC0185E30E943C1F882359F08091FC014C
:1040100085FB222720F991E0922790FB85F9809378
:10402000FC0181E30E943C1F882359F08091FC0130
:1040300086FB222720F991E0922790FB86F9809356
:10404000FC0181E10E943C1F882359F08091FC0112
:1040500087FB222720F991E0922790FB87F9809334
:10406000FC018091FC010E94B2208091FC0187FB41
:10407000882780F980930D0187E20E943C1FC82F9A
:104080008EE10E943C1F8111C2608FE10E943C1FA3
:104090008111C46080E20E943C1F8111C86081E2EE
:1040A0000E943C1F8111C06182E20E943C1F81116D
:1040B000C06283E20E943C1F8111C06484E20E94BE
:1040C0003C1F882311F0C06802C0CC2329F08C2F3C
:1040D0000E94A9206C2F03C00E94A520682F70E0C9
:1040E00080E090E0CF910C94391BCF9108956DEE54
:1040F0007EEF80E090E00E94E32660E082E090E0C6
:104100000E94D12660E083E090E00E94D12660E02A
:1041100084E090E00E94D12660E085E090E00C947D
:10412000D12680E090E00E94CB2621E08D3E9E4F7C
:1041300009F020E0822F089582E090E00C94C326DD
:10414000682F82E090E00C94D12683E090E00C94FC
:10415000C326682F83E090E00C94D12684E090E0A1
:104160000C94C326682F84E090E00C94D1268091B3
:10417000E40180FF0BC06091130185E0689FB001EE
:10418000112475956795759567952BC081FF09C0BA
:104190006091130185E0689FB001112475956795C2
:1041A00020C082FF07C06091130185E0689FB001C5
:1041B000112417C09091E5019923D1F0609112016B
:1041C000961788F72091130185E0289F900111240C
:1041D000929FA001939F500D112470E0CA010E948C
:1041E00095266038710540F46115710539F002C0FB
:1041F00065E070E0862F08958FE7089581E00895C7
:104200008091E40180FF08C06091110170E0759514
:1042100067957595679521C081FF06C06091110172
:1042200070E07595679519C082FF04C06091110117
:1042300070E010C09091E5019923C1F060911001E8
:104240009617A0F780911101899FC001112470E099
:104250000E9495266038710528F46115710521F0DA
:10426000862F08958FE7089581E0089561E070E05A
:10427000F4CF803F21F40E94B720819504C0813F94
:1042800029F40E94B7208093E8010895823F21F429
:104290000E94B720819504C0833F29F40E94B72073
:1042A0008093E7010895893F19F40E94002105C019
:1042B0008A3F31F40E94002181958093E90108959D
:1042C0008B3F21F40E940021819504C08C3F29F48A
:1042D0000E9400218093EA010895843F21F4809197
:1042E000E601816017C0853F21F48091E60182607C
:1042F00011C0863F21F48091E60184600BC0873FA6
:1043000021F48091E601886005C0883F31F48091F6
:10431000E60180618093E60108958D3F21F480914C
:10432000E40181600BC08E3F21F48091E401826042
:1043300005C08F3F29F48091E40184608093E401FB
:104340000895803F39F48091E80187FF6CC0109296
:10435000E80169C0813F29F48091E8011816BCF397
:1043600062C09091E701823F29F497FF5CC01092F0
:10437000E70159C0833F19F41916CCF354C0893FA3
:1043800041F48091E90118160CF04DC01092E9013A
:104390004AC08A3F29F48091E90187FF44C0F6CFE3
:1043A0008B3F39F48091EA0187FF3DC01092EA010A
:1043B0003AC08C3F29F48091EA011816BCF333C04F
:1043C000843F21F48091E6018E7F17C0853F21F460
:1043D0008091E6018D7F11C0863F21F48091E60136
:1043E0008B7F0BC0873F21F48091E601877F05C05A
:1043F000883F31F48091E6018F7E8093E60113C0FF
:104400008D3F21F48091E4018E7F0BC08E3F21F41B
:104410008091E4018D7F05C08F3F29F48091E401F4
:104420008B7F8093E4018091E70181110EC0809120
:10443000E80181110AC08091E901811106C08091D3
:10444000EA01811102C01092E501089586EE91E023
:104450000E94F7120E94911E9093E3018093E20163
:1044600008951F93CF93DF938091E2019091E30130
:104470000E949D1EAC019091E501992321F02091AD
:10448000140130E006C0209115018AE0289F9001B8
:1044900011244217530708F486C08091E701C091A8
:1044A000E801D091E9011091EA01811107C0C11121
:1044B00076C0D11174C0111172C075C09F3F19F040
:1044C0009F5F9093E501181624F40E94B720809313
:1044D000E7018091E70187FF05C00E94B720819521
:1044E0008093E7011C1624F40E94B7208093E80112
:1044F0008091E80187FF05C00E94B72081958093D5
:10450000E8016091E701662339F1C091E801CC230D
:1045100019F1772767FD7095872F972F0E94A625A1
:1045200023E333E343E35FE30E940A260E947325FB
:104530006093E7016C2F772767FD7095872F972F82
:104540000E94A62523E333E343E35FE30E940A26A8
:104550000E9473256093E8011D1624F40E94002137
:104560008093E9018091E90187FF05C00E94002145
:1045700081958093E901111624F40E940021809313
:10458000EA018091EA0187FF05C00E940021819520
:104590008093EA01DF91CF911F910C9426229F3FD7
:1045A00009F08ECF96CFDF91CF911F910895E6EE5F
:1045B000F1E085E0DF011D928A95E9F71092E501AF
:1045C0001092E4010895833081F128F4813059F08C
:1045D0008230D1F00895853009F449C0B8F18630B1
:1045E00009F456C0089580911501262F30E0280F58
:1045F000311D2F3F310524F4680F60931501089594
:104600008FEF80931501089580911401262F30E0DB
:10461000280F311D2F3F310524F4680F60931401DA
:1046200008958FEF80931401089580911301262F30
:1046300030E0280F311D2F3F310524F4680F6093BF
:10464000130108958FEF8093130108958091120153
:10465000262F30E0280F311D2F3F310524F4680F3D
:104660006093120108958FEF809312010895809155
:104670001101262F30E0280F311D2F3F310524F482
:10468000680F6093110108958FEF809311010895D1
:1046900080911001262F30E0280F311D2F3F31056A
:1046A00024F4680F6093100108958FEF8093100138
:1046B0000895833011F128F4813049F0823091F06F
:1046C0000895853081F120F18630C1F108958091FF
:1046D0001501681720F4861B809315010895109228
:1046E0001501089580911401681720F4861B8093AA
:1046F0001401089510921401089580911301681710
:1047000020F4861B809313010895109213010895DD
:1047100080911201681720F4861B8093120108957E
:1047200010921201089580911101681720F4861BE0
:104730008093110108951092110108958091100144
:10474000681720F4861B80931001089510921001C1
:1047500008950F931F938D3109F46BC008F03FC08B
:104760008E3009F47FC0C0F4873009F469C068F462
:10477000863009F0B1C08091DC01817F8E7F80930B
:10478000DC0181E08093EC01A8C0883009F4A2C06C
:104790008B3009F49FC0A0C0863109F49BC078F427
:1047A000803109F472C0813109F096C00E947917F6
:1047B00090910D0181E0892780930D018BC0893193
:1047C00009F488C08B3109F087C08091DC0181FB3E
:1047D000222720F991E0922790FB81F94CC0853384
:1047E00009F470C048F4873209F46CC008F459C069
:1047F000893209F467C070C0833438F48A3308F012
:104800004EC0883309F466C067C0833409F45AC0C7
:10481000883409F061C00E9479170FEF13ED20E38F
:10482000015010402040E1F700C000000E94EC1E43
:1048300051C00E942D250E94E0120E94D90B4AC04F
:104840009091DC01892F8095817080FB90F929F08F
:10485000966098609093DC0140C0997F977F909319
:10486000DC0138C08091DC0182FB222720F991E035
:10487000922790FB82F98093DC01992359F1809172
:10488000DC0181608093DC0125C08091DC0183FB29
:10489000222720F991E0922790FB83F9ECCF8953EE
:1048A00001C08D5141E050E060E070E08A019B0161
:1048B00004C0000F111F221F331F8A95D2F7C901B0
:1048C000B80104C061E070E080E090E00E94391B14
:1048D0000E94791781E001C080E01F910F91089537
:1048E00080E0089580E00895CF93C82F8091EC0177
:1048F000813079F018F08230E9F187C0E0910E0143
:10490000F0910F018081813169F0823209F07FC01E
:1049100009C0E0910E01F0910F018081813111F009
:10492000823261F48C2F0E947024811104C08C2F7C
:104930000E94A9231DC081E090E01AC08C2F0E9424
:104940007224811114C0C43179F048F4CB3079F06D
:10495000C03109F060C082E08093EC0108C0C93228
:1049600019F0C83321F057C01092EC0154C081E017
:10497000817053C0C93289F118F5C43171F1A8F4BE
:10498000C73009F046C08AE08093150194E1909306
:10499000140193E0909313018093120188E08093B7
:1049A000110188E28093100134C0CE51C63088F5E1
:1049B000EC2FF0E0E65DFE4F80818093EB0129C093
:1049C000CE34E9F020F4CB3421F56AE013C0C135D0
:1049D00079F0C235F1F461E00DC08091EB018823DC
:1049E00019F01092EB0115C081E08093EC0115C025
:1049F00061E006C08091EB010E94E3220AC06AE0F8
:104A00008091EB010E94592304C01092EC0180E0D8
:104A100004C081E002C080E0ABCFCF910895E1E80F
:104A2000F0E08081886080838081816080838FB79F
:104A3000F89493E09093890090ED909388008FBF55
:104A40000895EFE6F0E08081826080830895EFE6CC
:104A5000F0E080818D7F80830895EFE6F0E0908123
:104A600082E08927808308951F920F920FB60F92DC
:104A700011242F933F934F935F936F937F938F9363
:104A80009F93AF93BF93EF93FF938091ED0190912C
:104A9000EE0101969093EE018093ED01811103C028
:104AA00082E00E94D90BE091EE01E695E695F0E0F8
:104AB000E65BF74FE4918091ED018E1303C080E037
:104AC0000E94D90BFF91EF91BF91AF919F918F9170
:104AD0007F916F915F914F913F912F910F900FBEFA
:104AE0000F901F90189504D06894B1118DC008954F
:104AF00070D088F09F5790F0B92F9927B751A0F048
:104B0000D1F0660F771F881F991F1AF0BA95C9F761
:104B100012C0B13081F077D0B1E0089574C0672F32
:104B2000782F8827B85F39F0B93FCCF38695779511
:104B30006795B395D9F73EF49095809570956195FA
:104B40007F4F8F4F9F4F0895E89409C097FB3EF425
:104B500090958095709561957F4F8F4F9F4F9923CA
:104B6000A9F0F92F96E9BB279395F6958795779548
:104B70006795B795F111F8CFFAF4BB0F11F460FF08
:104B80001BC06F5F7F4F8F4F9F4F16C0882311F060
:104B900096E911C0772321F09EE8872F762F05C074
:104BA000662371F096E8862F70E060E02AF09A950F
:104BB000660F771F881FDAF7880F9695879597F904
:104BC000089557FD9058440F551F59F05F3F71F0FD
:104BD0004795880F97FB991F61F09F3F79F0879564
:104BE0000895121613061406551FF2CF4695F1DFED
:104BF00008C0161617061806991FF1CF869571057D
:104C0000610508940895E894BB2766277727CB01B0
:104C100097F908950BD078C069D028F06ED018F0BD
:104C2000952309F05AC05FC01124EECFCADFA0F36C
:104C3000959FD1F3950F50E0551F629FF001729F31
:104C4000BB27F00DB11D639FAA27F00DB11DAA1F50
:104C5000649F6627B00DA11D661F829F2227B00D9D
:104C6000A11D621F739FB00DA11D621F839FA00D28
:104C7000611D221F749F3327A00D611D231F849F78
:104C8000600D211D822F762F6A2F11249F575040CF
:104C90008AF0E1F088234AF0EE0FFF1FBB1F661F6A
:104CA000771F881F91505040A9F79E3F510570F023
:104CB00014C0AACF5F3FECF3983EDCF3869577955E
:104CC0006795B795F795E7959F5FC1F7FE2B880F1E
:104CD000911D9695879597F9089597F99F6780E8B4
:104CE00070E060E008959FEF80EC089500240A943E
:104CF0001616170618060906089500240A941216B7
:104D00001306140605060895092E0394000C11F4E9
:104D1000882352F0BB0F40F4BF2B11F460FF04C096
:104D20006F5F7F4F8F4F9F4F089597FB072E16F4AD
:104D3000009407D077FD09D00E94AF2607FC05D06C
:104D40003EF4909581959F4F0895709561957F4FA2
:104D50000895EE0FFF1F0590F491E02D0994AA1B12
:104D6000BB1B51E107C0AA1FBB1FA617B70710F056
:104D7000A61BB70B881F991F5A95A9F78095909588
:104D8000BC01CD010895F999FECF92BD81BDF89A7D
:104D9000992780B50895A8E1B0E042E050E00C9476
:104DA000EB26262FF999FECF92BD81BDF89A019787
:104DB00000B4021639F01FBA20BD0FB6F894FA9A63
:104DC000F99A0FBE08950196272F0E94D2260C94BF
:104DD000D126DC01CB01FC01F999FECF06C0F2BD62
:104DE000E1BDF89A319600B40D9241505040B8F7A9
:064DF0000895F894FFCFC6
:104DF6000220DB0B690C460C120CDE0B0101C9010B
:104E060028080A03140A3F4D36390B08BE078807DF
:104E16004F07E206FB0614072D07010203040506E9
:044E26000708090070
:00000001FF
